:020000020000FC
:100000000FC079C086C088C088C088C083C083C044
:0400100087C085C060
:10002000F89403E208BB0DE107BBF0E0E0E600E076
:100030000193E03AE9F70EE90DBF00E810E006BDD4
:1000400016BD00E00BBF00E009BF00E005BB00E605
:100050000ABF0EE008BF02E005BF00E002BF00E0FB
:100060000FBD00E003BF00E006BF00E009BD00E0F7
:1000700008BD00E007B900E003B900E006B900E000
:1000800004BB00E808B9A89504B7077F04BF01B511
:10009000006101BD0EE401BD00E40BBF00E009BF3B
:1000A000D2E1C0E5F5E0ECED05E0502E00EA402E8F
:1000B00090E07894A8950DE107BB90FFFBCF9E7F61
:1000C000132D022D37E028E0021B130B009510952D
:1000D00020E00894021F121F37E028E0020F131FD0
:1000E000D12FC02FC09A000000000000000021970F
:1000F000D1F7C098DFCFFFB6B0E0A0E0B19904C05F
:100100001196B4FD04C0FACF3B2E2A2E9160FFBE9B
:100110001895189518951895189518951895189577
:1001200018954F935F936F936627442711232AF402
:10013000439500951095061F161F33232AF4439507
:1001400020953095261F361F40FB0FD046F40095B2
:10015000109540955095061F161F461F561F242FB9
:10016000352F6F915F914F910895551B441B61E1AD
:1001700010F4420F531F57954795179507956A95A9
:04018000B9F708952E
:00000001FF
